:100000002F29A0007F39201B803C0920A01B003C29
:1000100008008A01820700340334063409340C34A2
:1000200010341334163419341C341F34223425345C
:1000300028342B342E3431343334363439343C3490
:100040003F3441344434473449344C344E345134D1
:100050005334553458345A345C345E34603462342A
:100060006434663468346A346B346D346F3470349D
:1000700071347334743475347634783479347A3432
:100080007A347B347C347D347D347E347E347E34EB
:100090007F347F347F347F349620B4000408B60068
:1000A0000800A4002508A402031CA5032708A60233
:1000B000031CA7033709A2003509A300A20A0319EC
:1000C000A30A4130A900AC01AD01AE01AF01A80106
:1000D000360884003409932084132B212408AC07AC
:1000E0000318AD0A2508AD072608AE070318AF0AA6
:1000F0002708AF072D080120803EA1002F0801200E
:10010000803EA107210CA80700083404031C340614
:100110008000290303194130A9000319A20A031919
:10012000A30F6D282A29841780052A29A8000530E5
:10013000A8190530840000308A0028080739820792
:100140000134023404340834103420344034803410
:100150000F39A00083161F088F3930389F00831293
:100160000310A00DA00D1F08C139200401389F0005
:100170000030A1003230E3209F149F18BD281E08D4
:10018000A10083161E082A2983169B001C141A0836
:100190002A2983169A001C1555309D00AA309D000F
:1001A0009C149C18D1281C112A29A301A200FF30FD
:1001B000A207031CA307031C2A290330A100E63071
:1001C000E320D728A101FC3EA000A109031CEE28D2
:1001D000FF300000A0070318E928A0076400A10F62
:1001E000E8280800A2000230FD28A2000130FD2806
:1001F000A2000630FD28A2000530A8002308210235
:10020000031D0429220820020430031801300319B9
:1002100002302805031DFF302A290038031DFF3056
:100220000405031DFF302A291030A800A101A001F8
:10023000A70CA60C031C22292208A00723080318D8
:10024000230FA107A10CA00CA50CA40CA80B182926
:1002500024082A29831303138312640008008930B9
:100260009F00E701FF30B800DE01DF010230A82067
:10027000DA002108DB00DC01DD015A08A0005B0880
:10028000A100A3012530F820031D47294A210A3087
:10029000D52036295A08A0005B08A1000330A3002E
:1002A0009230F520E0005A08A0005B08A10003305E
:1002B000A300FF30F820E2006008840062080D21EE
:1002C000E200E3005E08A0005F08A100A301003087
:1002D000F220E40062086304840064080D21E40055
:1002E000E50064006408650403197A290130E6001A
:1002F000AA2625265A08A0005B08A1000330A30007
:100300009230F520E0005A08A0005B08A1000330FD
:10031000A300FF30F820E2006008840062080D218D
:10032000E200E3005E08A0005F08A100A301013025
:10033000F220E40062086304840064080D21E400F4
:10034000E5006400640865040319A9290130E6008A
:1003500097265A08A0005B08A1000330A30049308B
:10036000F520E0005A08A0005B08A1000330A300BC
:100370009230F820E2006008840062080D21E2005B
:10038000E3005E08A0005F08A100A3010030F22096
:10039000E40062086304840064080D21E400E500C1
:1003A0006400640865040319D9290230E600AA260E
:1003B00025265A08A0005B08A1000330A30049309D
:1003C000F520E0005A08A0005B08A1000330A3005C
:1003D0009230F820E2006008840062080D21E200FB
:1003E000E3005E08A0005F08A100A3010130F22035
:1003F000E40062086304840064080D21E400E50061
:100400006400640865040319082A0230E600972690
:100410005A08A0005B08A1000230A300FF30F520BD
:10042000E0005A08A0005B08A1000330A300493097
:10043000F820E2006008840062080D21E200E30079
:100440005E08A0005F08A100A3010030F220E400D4
:1004500062086304840064080D21E400E500640080
:10046000640865040319382A0330E600AA26252605
:100470005A08A0005B08A1000230A300FF30F5205D
:10048000E0005A08A0005B08A1000330A300493037
:10049000F820E2006008840062080D21E200E30019
:1004A0005E08A0005F08A100A3010130F220E40073
:1004B00062086304840064080D21E400E500640020
:1004C000640865040319672A0330E60097265A0872
:1004D000A0005B08A1000230A300B630F520E000C8
:1004E0005A08A0005B08A1000230A300FF30F820EA
:1004F000E2006008840062080D21E200E3005E086B
:10050000A0005F08A100A3010030F220E40062080F
:100510006304840064080D21E400E50064006408BD
:1005200065040319972A0430E600AA2625265A08EE
:10053000A0005B08A1000230A300B630F520E00067
:100540005A08A0005B08A1000230A300FF30F82089
:10055000E2006008840062080D21E200E3005E080A
:10056000A0005F08A100A3010130F220E4006208AE
:100570006304840064080D21E400E500640064085D
:1005800065040319C62A0430E60097265A08A0001D
:100590005B08A1000230A3006D30F520E0005A088E
:1005A000A0005B08A1000230A300B630F820E200F2
:1005B0006008840062080D21E200E3005E08A000EC
:1005C0005F08A100A3010030F220E4006208630488
:1005D000840064080D21E400E500640064086504FB
:1005E0000319F62A0530E600AA2625265A08A00097
:1005F0005B08A1000230A3006D30F520E0005A082E
:10060000A0005B08A1000230A300B630F820E20091
:100610006008840062080D21E200E3005E08A0008B
:100620005F08A100A3010130F220E4006208630426
:10063000840064080D21E400E5006400640865049A
:100640000319252B0530E60097265A08A0005B0801
:10065000A1000230A3002530F520E0005A08A000D8
:100660005B08A1000230A3006D30F820E2006008B2
:10067000840062080D21E200E3005E08A0005F082C
:10068000A100A3010030F220E400620863048400AA
:1006900064080D21E400E5006400640865040319A2
:1006A000552B0630E600AA2625265A08A0005B082E
:1006B000A1000230A3002530F520E0005A08A00078
:1006C0005B08A1000230A3006D30F820E200600852
:1006D000840062080D21E200E3005E08A0005F08CC
:1006E000A100A3010130F220E40062086304840049
:1006F00064080D21E400E500640064086504031942
:10070000842B0630E60097265A08A0005B08A1005B
:100710000130A300DB30F520E0005A08A0005B08A0
:10072000A1000230A3002530F820E2006008840018
:1007300062080D21E200E3005E08A0005F08A1004E
:10074000A3010030F220E40062086304840064081E
:100750000D21E400E5006400640865040319B42B6E
:100760000730E600AA2625265A08A0005B08A1004B
:100770000130A3009130F520E0005A08A0005B088A
:10078000A1000130A300DB30F820E2006008840003
:1007900062080D21E200E3005E08A0005F08A100EE
:1007A000A3010030F220E4006208630484006408BE
:1007B0000D21E400E5006400640865040319E42BDE
:1007C0000830E600AA2625265A08A0005B08A100EA
:1007D0000130A3004930F520E0005A08A0005B0872
:1007E000A1000130A3009130F820E20060088400ED
:1007F00062080D21E200E3005E08A0005F08A1008E
:10080000A3010030F220E40062086304840064085D
:100810000D21E400E5006400640865040319142C4C
:100820000930E600AA2625265A08A0005B08A10088
:100830000130A3000030F520E0005A08A0005B085A
:10084000A1000130A3004930F820E20060088400D4
:1008500062080D21E200E3005E08A0005F08A1002D
:10086000A3010030F220E4006208630484006408FD
:100870000D21E400E5006400640865040319442CBC
:100880000A30E600AA2625265A08A0005B08A10027
:10089000A301B630F520E0005A08A0005B08A100D3
:1008A0000130A3000030F820E200600884006208F4
:1008B0000D21E200E3005E08A0005F08A100A30193
:1008C0000030F220E40062086304840064080D2113
:1008D000E400E5006400640865040319732C0B3020
:1008E000E600AA2625265A08A0005B08A100A3015D
:1008F0006E30F520E0005A08A0005B08A100A301BB
:10090000B630F820E2006008840062080D21E200A1
:10091000E3005E08A0005F08A100A3010030F22000
:10092000E40062086304840064080D21E400E5002B
:100930006400640865040319A12C0C30E600AA26A3
:1009400025265A08A0005B08A100A3012530F52048
:10095000E0005A08A0005B08A100A3016E30F82057
:10096000E2006008840062080D21E200E3005E08F6
:10097000A0005F08A100A3010030F220E40062089B
:100980006304840064080D21E400E5006400640849
:1009900065040319CF2C0D30E600AA262526023067
:1009A000A820DA002108DB00DC0A0319DD0A5C0854
:1009B000A0005D08A100A301C830F520E0005A089E
:1009C000A0005B08A100A3012530F520E20060082B
:1009D000840062080D21E200E3005A08A0005B08D1
:1009E000A100A3016E30F820E400620863048400D3
:1009F00064080D21E400E50064006408650403193F
:100A0000022DA8275E08A0005F08A100A301003006
:100A1000FB20031D192E5C08A0005D08A100A301A6
:100A2000C830F520E0005A08A0005B08A1000330A0
:100A3000A3009230F520E2006008840062080D21D6
:100A4000E200E3005A08A0005B08A1000330A30005
:100A5000FF30F820E40062086304840064080D217C
:100A6000E400E5006400640865040319382D3726A6
:100A70005C08A0005D08A100A301C830F520E000DB
:100A80005A08A0005B08A1000330A3004930F520FC
:100A9000E2006008840062080D21E200E3005A08C9
:100AA000A0005B08A1000330A3009230F820E4000E
:100AB00062086304840064080D21E400E50064001A
:100AC000640865040319652D37265C08A0005D08DD
:100AD000A100A301C830F520E0005A08A0005B087F
:100AE000A1000230A300FF30F520E200600884007E
:100AF00062080D21E200E3005A08A0005B08A10093
:100B00000330A3004930F820E40062086304840045
:100B100064080D21E400E50064006408650403191D
:100B2000922D37265C08A0005D08A100A301C83003
:100B3000F520E0005A08A0005B08A1000230A300E5
:100B4000B630F520E2006008840062080D21E20062
:100B5000E3005A08A0005B08A1000230A300FF30A8
:100B6000F820E40062086304840064080D21E400B6
:100B7000E5006400640865040319BF2D37265C088E
:100B8000A0005D08A100A301C830F520E0005A08CC
:100B9000A0005B08A1000230A3006D30F520E20048
:100BA0006008840062080D21E200E3005A08A000FA
:100BB0005B08A1000230A300B630F820E400620810
:100BC0006304840064080D21E400E5006400640807
:100BD00065040319EC2D37265C08A0005D08A10010
:100BE000A301C830F520E0005A08A0005B08A1006E
:100BF0000230A3002530F520E2006008840062087E
:100C00000D21E200E3005A08A0005B08A1000230B9
:100C1000A3006D30F820E4006208630484006408D7
:100C20000D21E400E5006400640865040319192E31
:100C300037260A30D5205A08A0005B08A100A3017E
:100C40002530F520031DCF2C080064006708203CE8
:100C5000031D2B2E08006708383E840066088000BC
:100C6000E70A6708383E8400FF308000080064000F
:100C7000203067020318482EFF306707E000FF307E
:100C80000318013EE1006008383E8400FF30800018
:100C9000E701FF306607E000FF300318013EE10086
:100CA0002130A600A7016008A2006108A30014215A
:100CB000E9006708383E84000008E000640060082E
:100CC000FF3C031D892E690883169B00FF308312A9
:100CD000C920E701FF30B80000304C20E830B700F1
:100CE0000330B5000630A700A500A430A6005120AF
:100CF0000230A820DA002108DB000A30D5205A088B
:100D0000A0005B08A100A3012530F520031D782E6B
:100D100008006708383E84000008E0006908831670
:100D20009B0083126008C920E70AE90A592EFF30A8
:100D30006607E000FF300318013EE1002130A60005
:100D4000A7016008A2006108A3001421E800680858
:100D5000C420E60064006608FF3C031DB02E0800B6
:100D600064006608013C031DC22E00304C204B304D
:100D7000B700B5018430A6000330A7000230A500FB
:100D8000BC30512064006608023C031DD42E0030A4
:100D90004C204B30B700B5014C30A6000430A70002
:100DA0000230A500BC30512064006608033C031DDE
:100DB000E62E00304C204B30B700B5014C30A60079
:100DC0000430A7000330A500843051206400660879
:100DD000043C031DF82E00304C204B30B700B50109
:100DE0001430A6000530A7000230A500BC30512009
:100DF00064006608053C031D0A2F00304C204B3070
:100E0000B700B5011430A6000530A7000330A500D7
:100E10008430512064006608063C031D1C2F0030FE
:100E20004C204B30B700B5011430A6000530A700A8
:100E30000430A5004C30512064006608073C031DB7
:100E40002E2F00304C204B30B700B501DC30A6000F
:100E50000530A7000230A500BC30512064006608B0
:100E6000083C031D402F00304C204B30B700B5012B
:100E7000DC30A6000530A7000330A50084305120E7
:100E800064006608093C031D522F00304C204B3093
:100E9000B700B501DC30A6000530A7000430A5007E
:100EA0004C305120640066080A3C031D642F00305A
:100EB0004C207830B700B501A430A6000630A7005A
:100EC0000430A5004C305120640066080B3C031D23
:100ED000762F00304C204B30B700B501DC30A60037
:100EE0000530A7000530A5001430512064006608C5
:100EF0000C3C031D882F00304C204B30B700B5014F
:100F0000A430A6000630A7000530A500DC30512033
:100F1000640066080D3C031D992F00304C20E8301A
:100F2000B7000330B5000A30A700A5002830A6009E
:100F300051205E08A0005F08A100A3010030FB2043
:100F4000031DA32F0800E80A4B30D520A72E080068
:100F50005E08A0005F08A100A3010130FB20031D73
:100F6000CD2FDE01DF01DC01DD0100304C204B30F4
:100F7000B700B5010630A700A500A430A600512097
:100F800000304C204B30B700B5010530A700A5005C
:100F90001430A60051200800F52F5E08A0005F085D
:100FA000A100A3010030FB20031DF52F0130DE005E
:100FB000DF01DC01DD0100304C204B30B700B50112
:100FC0000530A700A5001430A600512000304C20A9
:100FD0004B30B700B5010630A700A500A430A6002D
:0C0FE0005120E701FF30B80008000800B5
:02400E00EA3096
:00000001FF
